:0300000002000EED
:0300030002019F58
:20000B0002019675811BD2AFD2A91201A280FE12001B80FBC82581C822C92581C97A002228
:20002B00D083D082CF2581F581CFC082C08322CF2581F581CF22FBE493CB22FCE493FB7492
:20004B000193CC22FAE493F9740193CA2229F9E5F03AFA227C00CB30E7011CCB2275F0009B
:20006B0030E70215F022FDE493FF7401934F7004A3A3800C740293B50510740393B5F00A99
:20008B00E493C0E0740193C0E022A3A3A3A380D7FEEBA4FD8EF0ECA4FCEB8EF0A4C5F02C0F
:2000AB002DC5F02211B58EF0ED22C002C001AAF0F97E007D007F11C3E933F9EA33FADF0867
:2000CB00F5F0E9D001D00222ED33FDEE33FEC3ED9BF5F0EE9C40E0ADF0FED380DBBB0001E7
:2000EB0022C333C5F033C5F0DBF722BB000122C3C5F013C5F013DBF722240280022401C595
:20010B00F03400C5F022C394028003C39401C5F09400C5F0223116F4C5F0F4C5F02245F095
:20012B007022042231784024801A3178401E7014801A3178400E7014800A3178500E8004A0
:20014B00318C6008E4F5F022318C60F8E4F5F00422318C40F780ED318C40F170E780ED313C
:20016B008C40E170E780DD318C50E180D7C39BC5F09C20E70720D207C345F02220D2F9D340
:20018B0022C5F0C39C7003E5F09B22758CDC758A000508320508327400F508740075F00075
:2001AB00F50985F00A740075F000F51685F017748075F025C0E0C0F0120D7F15811581129D
:2001CB000DCE793B7A0EE98AF0F9AAF089828A83E493A3F5F0E493C5F0C0E0C0F0120DA2B3
:2001EB0015811581120369740175F00045F07003020237E5081200687B0112005F12012FF7
:20020B0045F060030201FE7400F5081202FD12038C1209B71203C61204671205581206EE78
:20022B0012076B1209D7120AC40201F2227F0912002B740078FC12001FF6740075F0000891
:20024B00F608A6F078FC12001FE61200687B0A12005F12015345F070030202AF801678FD38
:20026B0012001FE60886F012010818F608A6F012011680D0741175F000C0E0C0F0120DB68F
:20028B0015811581120DCE78FC12001FF608E60886F079F612002412005878FC12001FE699
:2002AB00F702026978FD12001FE60886F079F61200241200587400F778FD12001FE6088631
:2002CB00F07B007C0012014B45F070030202E274FF75F0FF0202F879F6120024E98AF0C0A5
:2002EB00E0C0F0120DE5158115810202F87FF702003AE59854011200687B0012005F12013A
:20030B005345F0700302031B120DCEF51102031F74FFF51122E59854011200687B0012002C
:20032B005F12015345F0700302033E120E30F51102034274FFF51122793F7A0EE98AF0F92E
:20034B00AAF089828A83E493A3F5F0E493C5F0C0E0C0F0120DA21581158112036922793D22
:20036B007A0EE98AF0F9AAF089828A83E493A3F5F0E493C5F0C0E0C0F0120DA21581158174
:20038B0022E5111200687B0A12005F12014B45F070030203C5793B7A0EE98AF0F9AAF0893F
:2003AB00828A83E493A3F5F0E493C5F0C0E0C0F0120DA21581158112036922E5111200682B
:2003CB007B6512005F12014B45F07003020466D2B3D2B4C2B5C2B6C2B7120BE1C2B3746491
:2003EB0075F000C0E0C0F0120B8F15811581740075F000F50985F00AE509850AF07B017CAA
:20040B000012012F45F070030204518012E509850AF0120108F50985F00A12011680D9C2B5
:20042B00A7740A75F000C0E0C0F0120B8F15811581D2A7740A75F000C0E0C0F0120B8F1592
:20044B00811581020418D2B3746475F000C0E0C0F0120B8F1581158112034322E5111200F0
:20046B00687B7712005F12014B45F07003020557D2B3C2B4D2B5D2B6D2B7D2A7120BE1E553
:20048B000F75F0007BFF7C0012014B45F0700302049FC2B3746475F000C0E0C0F0120B8F8E
:2004AB0015811581740075F000F51485F015740075F000F50985F00AE509850AF0AB16AC69
:2004CB001712015C45F070030205428012E509850AF0120108F50985F00A12011680D9740D
:2004EB001175F000C0E0C0F0120DB615811581E509850AF0F51285F013851290E51344804B
:20050B00F5A0120BE1120E30F580741375F000C0E0C0F0120DB615811581E5148515F02593
:20052B0080C5F03400C5F0F51485F015120B3E0030B2FD000204D8D2B3746475F000C0E085
:20054B00C0F0120B8F158115811203432205810581E5111200687B7212005F12014B45F021
:20056B00700302063B740075F000F51485F015E50E75F0007B727C0012014B45F0700CE599
:20058B000E75F0007B537C0012014B45F070030205A2C2B30205A4D2B3D2A7C2B4D2B5D2F7
:2005AB00B6D2B77431F50D740075F00078FD12001FF608A6F078FD12001FE60886F0AB166C
:2005CB00AC1712015C45F07003020638801678FD12001FE60886F012010818F608A6F0127D
:2005EB00011680D178FD12001FE60886F0F51285F013851290E5134480F5A0C2B5120BE102
:20060B007580FFE5148515F02580C5F03400C5F0F51485F015E580120068C0E0C0F012063B
:20062B004015811581D2B51206670205D9120343158115812278FB12001FE6F50BE50B75C8
:20064B00F0007B047C001200F6F50B12068A78FB12001FE6540FF50B12068A221203207B99
:20066B00137C0012014B45F070030206891203207B117C0012015345F0600302067822E587
:20068B000B75F0007B097C0012016A45F070030206B2E50B243775F000C0E0C0F0120DB62B
:2006AB00158115810206C4E50B243075F000C0E0C0F0120DB61581158122E5801200687BC1
:2006CB00FF12005F12015345F070030206ED7430F50DE51A851BF0120108F51A85F01B129B
:2006EB00011622E5111200687B6C12005F12014B45F0700302076AC2B3D2A7D2B4D2B5D2A8
:20070B00B6D2B7746475F000C0E0C0F0120B8F15811581120B3E740575F000C0E0C0F0128F
:20072B000B8F15811581C2B6C2B7120BE1120B3E740575F000C0E0C0F0120B8F1581158198
:20074B00C2B5D2B6C2B7120BE1120B3E740575F000C0E0C0F0120B8F15811581120343223D
:20076B00E5111200687B6312005F12014B45F070030207AF748175F00EC0E0C0F0E51485BB
:20078B0015F01201222401C5F03400C5F0C0E0C0F0740275F000120C2A1581158115811507
:2007AB008112034322D2B3740A75F000C0E0C0F0120B8F158115811207EEE50E75F0007BC9
:2007CB00FF7C0012014B45F070030207EDC2B3740A75F000C0E0C0F0120B8F158115811205
:2007EB0007EE22D2A7C2B4D2B5C2B6C2B7743175F000F51285F013851290E5134480F5A05F
:20080B00C2B5120BE17580FFE580F50ED2B5E5128513F0120108F51285F01312011685128C
:20082B0090E5134480F5A0C2B5120BE17580FFE580F50FD2B322058105811207B0E50E7516
:20084B00F0009008C8020071740075F010F51885F0190208F0740075F010F51885F01902C6
:20086B0008F0740075F020F51885F0190208F0740075F020F51885F0190208F0740075F080
:20088B0050F51885F0190208F0740075F050F51885F0190208F0740075F028F51885F0190E
:2008AB000208F0740075F030F51885F0190208F0740075F000F51885F0190208F0BB08FF65
:2008CB0000AE085300A108720094086500870855007A0862006D08520060086100530851E4
:2008EB00000000F008740075F000F51485F015740075F000F51A85F01BE50E75F0007B72CC
:20090B007C0012014B45F0700CE50E75F0007B537C0012014B45F0700302092CC2B30209E2
:20092B002ED2B3D2A7C2B4D2B5D2B6D2B77431F50D740075F00078FD12001FF608A6F07840
:20094B00FD12001FE60886F0AB18AC1912015C45F070030209B2801678FD12001FE60886EE
:20096B00F012010818F608A6F012011680D178FD12001FE60886F0F51285F013851290E596
:20098B00134480F5A0C2B5120BE17580FFE5148515F02580C5F03400C5F0F51485F015120C
:2009AB0006C5D2B50209631581158122E5111200687B7312005F12014B45F070030209D668
:2009CB00120238F51685F01712034322E5111200687B6712005F12014B45F07003020AC317
:2009EB00120841E50E75F0007BFF7C0012015345F07003020AB0749175F00EC0E0C0F0E5CC
:200A0B000E75F000C0E0C0F0740275F000120C2A1581158115811581E50F75F0007BFF7C3E
:200A2B000012014B45F07003020A4674A075F00EC0E0C0F0120DA215811581E50F75F00036
:200A4B007B057C0012014B45F07003020A6974A575F00EC0E0C0F0120DA21581158174A92E
:200A6B0075F00EC0E0C0F0E51A851BF0C0E0C0F0740275F000120C2A15811581158115814E
:200A8B0074BD75F00EC0E0C0F0E5168517F0C0E0C0F0740275F000120C2A1581158115819B
:200AAB001581020AC074D075F00EC0E0C0F0120DA21581158112034322E5111200687B7000
:200ACB0012005F12014B45F07003020B3D120841E50E75F0007B727C0012014B45F0700C1F
:200AEB00E50E75F0007B537C0012014B45F07003020B057455F510020B09E50EF51074E2FF
:200B0B0075F00EC0E0C0F0E51075F000C0E0C0F0E51A851BF0C0E0C0F0E5168517F0C0E057
:200B2B00C0F0740475F000120C2A7FF812002B12034322C2A7000000D2A722058105817423
:200B4B000075F00078FD12001FF608A6F078FD12001FE60886F07B087C0012012F45F070FB
:200B6B0003020B8A801678FD12001FE60886F012010818F608A6F012011680D1020B71155C
:200B8B008115812205810581740075F00078FD12001FF608A6F078FD12001FE60886F07870
:200BAB00F912001F860308860412012F45F07003020BDC801678FD12001FE60886F012015F
:200BCB000818F608A6F012011680CB120B46020BC0158115812205810581740075F0007807
:200BEB00FD12001FF608A6F078FD12001FE60886F07B017C0012012F45F07003020C258089
:200C0B001678FD12001FE60886F012010818F608A6F012011680D1020C0C158115812223DD
:200C2B00F42581F8868208868308E4FEFF93700122B42555A3E493B42D06430780A3E493DC
:200C4B00B4300343074024D0B40A00500CCE75F00AA42EFEA3E49380EDE493B46413E608E6
:200C6B0086F030F708430720120120A6F018F68003B4750543070A801CB4780543071080D7
:200C8B0014B46F0B430708800C120DBCA3809BB462624307027A00C004C005C006C007AB91
:200CAB000753031F7C00E60886F01200B5A6F018F6EDD007D006D005D0042430B43A00409D
:200CCB00022407C0E00AE645F070CCA902EF30E506742D120DBC0A120D60D0E0120DBCD9BD
:200CEB00F90808EF30E7A5EAC39E50A07420120DBC0A80F3B4630BAA01120D60E6120DBC01
:200D0B0080DFB4732BC082C08386820886837A00E4936004A30A80F88683188682120D6057
:200D2B00E493A36005120DBC80F6D083D08280B1B4691986017A00E76004090A80F9120DD5
:200D4B00608601E7609B120DBC0980F7F97A01120D60E980A8EE601B8FF020F716C002EA9F
:200D6B00C39E500D742030F6027430120DBC0A80EED0022278FB12001F8603088604748050
:200D8B0075F0701200B5120120758921F58DF58B7588597598522278FB12001F8682088647
:200DAB0083E4936034120DBCA380F678FB12001FE63099FDC299F599B40A1E740D80F2E4BA
:200DCB003098133098FDC298E5993099FDC299F599B40D02740A75F0002278FB12001F86EF
:200DEB0001E4FBFCFFE709B42D030FE709C39430B40A005012FA740A75F00012009B2AFBE4
:200E0B00E5F03400FC80E4EB8CF0DF030201202278FB12001FE63099FDC299F5992274FF02
:200E2B00F5F030980A3098FDC298E59975F00022410E780E7C0E0A20456173792D446F775A
:200E4B006E6C6F616465722056322E3220666F722041544D454C2038394335312F35322FA1
:200E6B0035352053383235322F533533000A203E000A206F6B000A2043484B53554D203D11
:200E8B002025303478000A20666F756E6420383943253278002D313256002D3556000A2075
:200EAB006E6F6E626C616E6B202575206279746573000A20627974657320636F756E7465D4
:200ECB0072202575000A204E6F7420666F756E642038394378780025782C25752C25750057
:00000001FF
